:100000000C94F5040C943C050C943C050C943C05B4
:100010000C943C050C943C050C943C050C943C055C
:100020000C943C050C943C050C94AE0D0C94800E85
:100030000C942A1C0C943C050C943C050C943C0537
:100040000C943C050C943C050C943C050C943C052C
:100050000C943C050C949E1C0C943C050C943C05A3
:100060000C943C050C943C050C943C050C943C050C
:100070000C943C050C943C050C943C050C943C05FC
:100080000C943C050C943C050C943C050C943C05EC
:100090000C943C050C943C050C943C050C943C05DC
:1000A0000C943C050C943C050C943C05ED0E0F0F94
:1000B000FD0F0F0FFD0F540F770FFD0FCC0FDF0F4C
:1000C0001913191346134613A113DD13D515D515AE
:1000D000F513D515F014F014AB15D515D515C115BC
:1000E000041607090B0A1D1B06198005141A0815AA
:1000F0001C171E1F202123222E26242D25273012D7
:10010000182F0C13280F0D340E33313638111037D9
:100110002B2C352A7F80807B79397A808080808083
:1001200080634F8080805053518080805852578028
:10013000808062595A5B5C5D5E5F80606180808018
:10014000808056808080668054808080805580804A
:100150000A0025303862003A200025303258000A63
:10016000722F632030313233343536370A005D0A5E
:100170000025303258005B0020002530325800281E
:1001800031290A002832290A002833290A00283494
:10019000290A000A0025303258006D303131305FB5
:1001A00072656376206572723A20000A002530324B
:1001B00058006D303131305F73656E642065727246
:1001C0003A20005B735D004B6579626F6172642059
:1001D00073746172742E0A0055534220636F6E6609
:1001E0006967757265642E0A005B575D005B535D3D
:1001F000005B525D005B445D005B435D0032034D7C
:1002000000300031003100300020006B00650079C3
:100210000062006F00610072006400200063006FE4
:10022000006E0076006500720074006500720000C8
:10023000000E0374002E006D002E006B002E0000D7
:10024000000403090409027400040100A032090437
:1002500000000103010100092111010001224000F9
:100260000705810308000A090401000103010200D7
:10027000092111010001224D000705820308000A2F
:1002800009040200010300000009211101000122FC
:1002900036000705830308000A090403000203006F
:1002A000000009211101000122220007058403201A
:1002B00000010705040320000112011001000000E5
:1002C00008EDFE10010101010200010631FF097471
:1002D000A1010975150026FF009520750881020906
:1002E00076150026FF00952075089102C0050109CA
:1002F00080A101850216810026B7001A81002AB765
:1003000000751095018100C0050C0901A10185034C
:10031000160100269C021A01002A9C027510950104
:100320008100C005010902A1010901A10005091907
:1003300001290515002501950575018102950175B5
:100340000381010501093009311581257F95027569
:1003500008810609381581257F95017508810605F4
:100360000C0A38021581257F950175088106C0C0E9
:1003700005010906A101050719E029E71500250176
:10038000950875018102950175088101050819011B
:1003900029059505750191029501750391010507E0
:1003A000190029FF150026FF00950675088100C079
:1003B0000A002530325820006B6579626F617264E3
:1003C0005F7265706F72743A20004C45443A202584
:1003D0003032580A00290A002575002F00257500C3
:1003E0005D280025640020002564002000256400AD
:1003F00020002564007C0025303258006D6F757335
:10040000656B6579205B62746E7C7820792076203C
:10041000685D287265702F61636C293A205B006DFE
:100420006B5F776865656C5F74696D655F746F5F3E
:100430006D6178203D2025640A006D6B5F776865EB
:10044000656C5F6D61785F7370656564203D202524
:10045000640A006D6B5F74696D655F746F5F6D61D9
:1004600078203D2025640A006D6B5F6D61785F73B5
:1004700070656564203D2025640A006D6B5F696EC0
:1004800074657276616C203D2025640A006D6B5F97
:1004900064656C6179203D2025640A006D6B5F778F
:1004A0006865656C5F74696D655F746F5F6D6178B9
:1004B000203D2025640A006D6B5F776865656C5F81
:1004C0006D61785F7370656564203D2025640A0066
:1004D0006D6B5F74696D655F746F5F6D6178203DF2
:1004E0002025640A006D6B5F6D61785F73706565D0
:1004F00064203D2025640A006D6B5F696E7465722F
:1005000076616C203D2025640A006D6B5F64656C2C
:100510006179203D2025640A000A00257500363ADD
:1005200020776865656C5F74696D655F746F5F6D7A
:1005300061783A20000A00257500353A2077686511
:10054000656C5F6D61785F73706565643A20000A61
:1005500000257500343A2074696D655F746F5F6DB6
:1005600061783A20000A00257500333A206D6178E1
:100570005F73706565643A20000A00257500323AA1
:1005800020696E74657276616C286D73293A20005B
:100590000A00257500313A2064656C6179282A319A
:1005A000306D73293A20000A092D2056616C75655B
:1005B00073202D0A004D3E004D25643E20003F0073
:1005C0007365742064656661756C740A00433E202F
:1005D0000077686572652064656C74613A206375A4
:1005E00072736F723D25642C20776865656C3D25BC
:1005F000640A53656520687474703A2F2F656E2EF7
:1006000077696B6970656469612E6F72672F7769AE
:100610006B692F4D6F7573655F6B6579730A000A9F
:10062000092D204D6F7573656B6579202D0A455333
:10063000432F713A09717569740A313A0964656C1E
:100640006179282A31306D73290A323A09696E744A
:10065000657276616C286D73290A333A096D617889
:100660005F73706565640A343A0974696D655F7417
:100670006F5F6D61780A353A09776865656C5F6D03
:1006800061785F73706565640A363A0977686565F5
:100690006C5F74696D655F746F5F6D61780A0A7075
:1006A0003A097072696E742076616C7565730A64BC
:1006B0003A097365742064656661756C74730A75B4
:1006C000703A092B310A646F776E3A092D310A703E
:1006D0006775703A092B31300A7067646F776E3A2C
:1006E000092D31300A0A7370656564203D20646508
:1006F0006C7461202A206D61785F73706565642079
:100700002A2028726570656174202F2074696D65D8
:100710005F746F5F6D6178290A003F004D3E2000D5
:10072000433E20004C25640A000A092D20436F6EC9
:10073000736F6C65202D0A4553432F713A0971750B
:1007400069740A6D3A096D6F7573656B65790A0096
:100750000A092D204D61676963202D0A643A0964F6
:10076000656275670A783A096465627567206D612C
:10077000747269780A6B3A096465627567206B6503
:1007800079626F6172640A6D3A0964656275672007
:100790006D6F7573650A763A0976657273696F6E67
:1007A0000A733A097374617475730A633A09636F63
:1007B0006E736F6C65206D6F64650A302D343A0975
:1007C0006C61796572302D34284631302D463429DC
:1007D0000A506175733A09626F6F746C6F6164657A
:1007E000720A003F0074696D65725F7265616433FF
:1007F0003228293A202530346C580A006B6579621A
:100800006F6172645F69646C653A2025580A006BF9
:100810006579626F6172645F70726F746F636F6C21
:100820003A2025580A00686F73745F6B6579626FB0
:100830006172645F6C65647328293A2025580A0048
:100840000A092D20537461747573202D0A004743E3
:10085000433A20342E392E32204156522D4C4942F3
:10086000433A20312E382E3073766E204156525F37
:10087000415243483A20617672350A004F5054493C
:100880004F4E533A204C554641204D4F5553454B02
:1008900045592045585452414B455920434F4E53DA
:1008A0004F4C4520434F4D4D414E44204B45594DF3
:1008B00041505F53454354494F4E20343039360A36
:1008C000004255494C443A20633766643566632DCF
:1008D0006469727479202830343A31393A353120DC
:1008E0005365702031332032303136290A005649A1
:1008F000443A2030784645454428742E6D2E6B2EA0
:1009000029205049443A20307830313130284D3058
:10091000313130206B6579626F61726420636F6E74
:1009200076657274657229205645523A20307830C7
:100930003130310A00444553433A20636F6E766587
:100940007274204D30313130206B6579626F617285
:100950006420746F205553420A000A092D20566501
:100960007273696F6E202D0A000A6D6F7573653A98
:10097000206F66660A000A6D6F7573653A206F6EA8
:100980000A000A6B6579626F6172643A206F66666D
:100990000A000A6B6579626F6172643A206F6E0AB1
:1009A000000A6D61747269783A206F66660A000AFF
:1009B0006D61747269783A206F6E0A000A6465622C
:1009C00075673A206F6E0A000A64656275673A209F
:1009D0006F66660A000A0A626F6F746C6F61646505
:1009E000722E2E2E2000433E200011241FBECFEF7A
:1009F000DAE0DEBFCDBF04B603FE27C08091D4018C
:100A00009091D501A091D601B091D7018730904B3C
:100A1000A740B04BD1F41092D4011092D50110929E
:100A2000D6011092D70114BE84B7877F84BF0FB65A
:100A3000F894A8958091600088618093600010927E
:100A400060000FBEE0E0F8E3099511E0A0E0B1E03E
:100A5000EAE1FAE402C005900D92A233B107D9F79A
:100A600021E0A2E3B1E001C01D92A43DB207E1F78D
:100A70000E94DD0A0C940B250C940000FF93EF9369
:100A8000E0913201F0913301309709F00995EF912F
:100A9000FF910895FC018591803011F0EFDFFBCFCD
:100AA0000895FF27E0E230E247FF0CC0419597FF31
:100AB00009C0EDE26095709580959095611D711D5E
:100AC000811D911D27FF02C0219530E350E2AA2726
:100AD000660F771F881F991FAA1FA41710F0A41B69
:100AE00063955A95A9F7AA3008F0A95FA05DAF9366
:100AF000F395611571058105910541F7ED3211F40A
:100B0000EF93F395F21718F43F93F395FBCF8F9182
:100B1000B5DFFA95E1F70895E991F9918591803073
:100B200021F0853219F0AADFF9CF089520E0E8948A
:100B300055915532C1F3503311F4689455915A339D
:100B400048F4505390F3220F022E220F220F200D53
:100B5000250FF4CF0EF4219589919991533619F30D
:100B6000533729F1533559F1BC0188279927E89467
:100B70005C3621F48991999168945591543639F4F1
:100B800046EF7EF077FF0DC08FEF9FEF0AC055371D
:100B90004AE039F0583540E121F0523642E009F0A0
:100BA0000895FF93EF937DDFEF91FF91B7CFFF9310
:100BB000EF93FC0181918030B9F360DFFBCFFF93AD
:100BC000EF9368DFF1CFDF93CF93CDB7DEB72596F4
:100BD000A3DFCF91DF9108950E94E106E4E3F1E005
:100BE0008EE08E0F11928E13FDCF84E391E09093EF
:100BF000430180934201569A5E9A2FEF89E698E16D
:100C0000215080409040E1F700C00000569A5E9865
:100C10000895CF93109244010E94FB07C82F8B3791
:100C200009F444C08F3F09F441C081E0809344013E
:100C30008C2F869586958695E0914201F09143012F
:100C40004C2F4770C7FF0EC08F70E80FF11D21E0D9
:100C500030E001C0220F4A95EAF7209580812823D1
:100C600020830BC0E80FF11D81E090E001C0880FE8
:100C70004A95EAF79081892B80838091B60180FFA5
:100C800017C086E791E00E944A051F92CF9381E743
:100C900091E09F938F930E94E3058EE691E00E947E
:100CA0004A050F900F900F900F9002C080E001C096
:100CB00081E0CF9108952091420130914301F901E3
:100CC000E80FF11D80810895EF92FF920F931F931B
:100CD000CF93DF938FE591E00E944A05C0E0D0E01A
:100CE0008AE5E82E81E0F82E02E511E0DF93CF934C
:100CF000FF92EF920E94E30587E591E00E944A058A
:100D0000E0914201F0914301EC0FFD1F80810E94B0
:100D1000BF1B1F928F931F930F930E94E30580E5E3
:100D200091E00E944A0521968DB79EB708960FB6AE
:100D3000F8949EBF0FBE8DBFCE30D105B9F6DF91BE
:100D4000CF911F910F91FF90EF900895569A81FFD8
:100D500002C05E9A08955E9808955198599A089530
:100D60005898509A08955098589A08955198599AB9
:100D700085E08A95F1F7000089B186958170089524
:100D8000CF93DF93EC010E94B606882341F02097B1
:100D900031F085E08A95F1F700002197F4CFCE017C
:100DA000DF91CF9108958B3741F08F3F41F0982F1D
:100DB0009F7796958078892B08958BE708958FEF1C
:100DC00008950E94AD060E94B3062FEF83ED90E3D5
:100DD000215080409040E1F700C000000895EF925C
:100DE000FF920F931F93CF93DF93E82E1092480149
:100DF0000E94AD060E94B006CAEFD0E088EE93E0F4
:100E00000E94C006892B21F42197C1F781E036C0EA
:100E100008E010E080E8F82E8AEF90E00E94C0061B
:100E2000892B11F483E02AC08F2D8E2129F00E9496
:100E3000B306C8ECD0E00AC00E94B006FACF2097F3
:100E400059F025E02A95F1F7000021970E94B60697
:100E50008823A9F3CD2B11F484E010C0F69401503F
:100E60001109D1F68FE891E00197F1F700C0000079
:100E70000E94AD060E94B30681E026C0809348011F
:100E800082EB91E00E944A05809148011F928F9366
:100E90008DEA91E09F938F930E94E3058BEA91E0A6
:100EA0000E944A059FEF29E688E19150204080404A
:100EB000E1F700C000000E94AD060E94B3060F904B
:100EC0000F900F900F9080E0DF91CF911F910F91C5
:100ED000FF90EF9008950F931F93CF93DF9310929D
:100EE0004801CAEFD0E088EE93E00E94C006892B4B
:100EF00021F42197C1F781E02FC0D8E0C0E0CC0FEA
:100F000088EC90E00E94C006892B11F482E024C096
:100F100008EC10E00E94B60681110AC00115110507
:100F200049F025E02A95F1F7000001501109F2CFB0
:100F3000012B11F483E010C05098589A85E08A95EF
:100F4000F1F700004899C160D150C9F60E94AD0682
:100F50000E94B3068C2F26C0809348018AE991E055
:100F60000E944A05809148011F928F9385E991E084
:100F70009F938F930E94E30583E991E00E944A05C5
:100F80009FEF29E688E1915020408040E1F700C0C2
:100F900000000E94AD060E94B3060F900F900F90C4
:100FA0000F908FEFDF91CF911F910F910895CF9305
:100FB00084E10E94EF060E946B07C82F8B37C1F0B7
:100FC0008091B60180FF0CC01F92CF938AE791E019
:100FD0009F938F930E94E3050F900F900F900F90B7
:100FE0008091B60180FF04C088E791E00E944A0525
:100FF0008C2FCF910895CF93DF9380914701882361
:1010000019F0109247017EC080914601882319F0A3
:101010001092460177C0C0914501CC2319F010927F
:10102000450103C00E94D707C82F8C2F8F778137C7
:10103000B1F0893709F061C00E94D707982F9F77D8
:101040009D3041F018F4953039F404C0913111F01D
:101050009B3111F487FD37C00E94D3063AC00E942D
:10106000D707982F9F77913719F0993721F041C012
:101070008093450142C00E94D707D82F8F778D30CB
:1010800041F018F4853081F504C0813111F08B31C5
:1010900059F5C7FF11C0D7FF0AC08EE891E00E9442
:1010A0004A058C2F0E94D306809346010BC089E825
:1010B00091E00E944A0521C0D7FF0DC084E891E06D
:1010C0000E944A058D2F0E94D306982F9066909318
:1010D0004701806417C08FE791E00E944A058D2F79
:1010E0000E94D30680660EC08D2F0E94D3068064B6
:1010F00002C00E94D306809347018C2FDF91CF91CD
:101100000C94D306DF91CF910895809154010895F6
:101110009FB7F89410924B019FBF9091CB019430F0
:1011200009F057C09091E9009F703091EC00232F97
:10113000217030FD20E8922B24E02093E9002091DB
:10114000EB0020FF43C02091EE0027FF3FC020911D
:101150004901222321F02091E80025FF37C0109299
:10116000490126E03091E80035FD15C03091CB01F2
:10117000343061F53091EB0035FD28C0215021F469
:1011800081E08093490122C0EFE9FFE03197F1F758
:1011900000C00000E7CF8093F1008091E80085FD5A
:1011A0000AC08091E80080FFFCCF8091E8008E7734
:1011B0008093E80006C08FB7F89421E020934B019C
:1011C0008FBF9F709093E90080E008959F70909387
:1011D000E9008FEF0895CF93DF9300D01F92CDB732
:1011E000DEB79C018091CB01843019F593E099839F
:1011F0003B832A839093E9008FEF9091E800815020
:1012000095FD06C095ED9A95F1F700008111F5CF97
:101210008091E80085FF0DC040E050E063E070E0A1
:10122000CE0101960E949E0B8091E8008E778093FC
:10123000E8000F900F900F90DF91CF910895CF931A
:10124000DF9300D01F92CDB7DEB72091CB012430C1
:1012500021F522E029839B838A8383E08093E90040
:101260008FEF9091E800815095FD06C095ED9A951D
:10127000F1F700008111F5CF8091E80085FF0DC0E6
:1012800040E050E063E070E0CE0101960E949E0BCA
:101290008091E8008E778093E8000F900F900F9078
:1012A000DF91CF9108952091CB012430F1F422E019
:1012B0002093E9002FEF3091E800215035FD06C062
:1012C00035ED3A95F1F700002111F5CF2091E800B6
:1012D00025FF0BC040E050E065E070E00E949E0BEF
:1012E0008091E8008E778093E8000895CF93DF9394
:1012F0002091CB01243039F521E02093E9002FEF34
:101300003091E800215035FD06C035ED3A95F1F7F2
:1013100000002111F5CF2091E80025FF14C0EC0159
:1013200040E050E068E070E00E949E0B8091E80091
:101330008E778093E80088E0FE01ACE4B1E0019094
:101340000D928A95E1F7DF91CF91089589EF91E0B1
:101350000E944A058091CA01811109C00E94330D83
:101360000E94900D8091E20084608093E2000895D5
:1013700085EF91E00E944A051092CA01089581EF1D
:1013800091E00C944A0520914A012F5F822F62E37D
:101390000E94D124992319F020934A0108951092B4
:1013A0004A0180914B01882371F18091CB018430F7
:1013B00041F58091E9008F702091EC00922F91709F
:1013C00020FD90E8892B94E09093E9009091EB0048
:1013D00090FF14C09091EE0097FF10C09091E8002C
:1013E00095FF03C01092F100F9CF9091E80090FFB3
:1013F00005C09091E8009E779093E8008F708093ED
:10140000E90010924B01089542E061EC81E00E94F6
:10141000AD0C42E061EC82E00E94AD0C42E061EC78
:1014200083E00E94AD0C42E261EC84E00C94AD0CD0
:101430008091CD01833009F453C030F4813071F0D4
:10144000823009F48CC008958A3009F478C08B305A
:1014500009F45EC0893009F09AC020C08091CC01A7
:10146000813A09F094C08091E800877F8093E8007A
:101470008091D0019091D101892B21F468E08CE416
:1014800091E003C060E080E090E070E00E94E90B32
:101490008091E8008B778093E80008958091CC01DB
:1014A000813209F074C08091D0019091D101892BD3
:1014B00009F06DC08091E800877F8093E8008091FB
:1014C000E80082FD05C08091CB018111F8CF5FC09B
:1014D0008091F100809354018091E8008B7753C094
:1014E0008091CC01813A09F052C08091D001909155
:1014F000D101892B09F04BC08091E800877F809350
:10150000E8008091E80080FFFCCF80910A0136C09E
:101510008091CC018132D9F58091D0019091D10197
:10152000892BA9F58091E800877F8093E8000E94CD
:10153000E20C8091CE0180930A010C94F615809103
:10154000CC01813221F58091E800877F8093E8000B
:101550000E94E20C8091CF01809355010895809103
:10156000CC01813AA1F48091E800877F8093E80064
:101570008091E80080FFFCCF809155018093F100BD
:101580008091E8008E778093E8000C94E20C089537
:101590000895089508958DEE91E00E944A050C94F7
:1015A000CA0A0E94E91B8091C901882329F00E9480
:1015B000141C81110C94880B089584B7877F84BF15
:1015C0000FB6F894A89580916000886180936000C0
:1015D000109260000FBE90E080E80FB6F894809300
:1015E0006100909361000FBE0E94C80A0E94A7107C
:1015F0000E94330D0E94900D8091E20084608093E0
:10160000E20088E898E00E94BA1B78948091CB01B0
:101610008430E1F788ED91E00E944A050E94A9100C
:1016200080E091E00E94151087EC91E00E944A054D
:101630000E94C90A8091CB01853039F483EC91E096
:101640000E944A050E94D10AF5CF0E94AD10F2CF48
:101650000C94281C89EE91E00E944A050C94280BFA
:10166000292F332723303105C9F064F421303105A7
:1016700081F02230310509F043C084E790E025E491
:1016800032E042C021323105F1F02232310541F120
:1016900037C082E190E029EB32E036C099278130F3
:1016A000910541F08230910541F0892B49F5E1E443
:1016B000F2E005C0E1E3F2E002C0EDEFF1E0849179
:1016C00090E09F0121C06430D8F4E62FF0E0EE0FE7
:1016D000FF1FE15EFE4F2081318189E090E014C060
:1016E000643070F470E0FB01EE0FFF1FE95EFE4F07
:1016F00020813181FB01ED5EFE4F808190E004C0CE
:1017000080E090E020E030E0FA013183208308950A
:1017100080E189BD82E189BD09B400FEFDCF8091E1
:10172000D8008F7D8093D8008091E0008260809304
:10173000E0008091E00081FDFCCF0895CF92DF9220
:10174000EF92FF920F931F93CF93DF93EC018B01E6
:101750006A010E94010D811133C0C114D10439F016
:10176000F60180819181081B190BC80FD91FE12C4C
:10177000F12C0115110519F18091E80085FD16C0C5
:101780008091E8008E778093E800C114D10449F07D
:10179000F60180819181E80EF91EF182E08285E0F8
:1017A0000FC00E94010D882321F30AC08991809304
:1017B000F10001501109FFEFEF1AFF0ADACF80E0C4
:1017C000DF91CF911F910F91FF90EF90DF90CF901D
:1017D00008952091D2013091D3012617370748F0A0
:1017E0006115710539F42091E8002E772093E80007
:1017F00001C0B90140E061157105A9F12091CB014B
:10180000222309F443C0253009F442C02091E800A6
:1018100023FD40C02091E80022FD32C02091E80065
:1018200020FFE9CF4091F3002091F20030E0342B0B
:10183000FC01CF016115710559F02830310540F4E4
:1018400081918093F100615071092F5F3F4FF1CF7B
:1018500041E02830310509F040E02091E8002E7782
:101860002093E800C8CF4111C9CF0AC08091CB01B5
:10187000882361F0853061F08091E80083FD0AC023
:101880008091E80082FFF2CF80E0089582E0089521
:1018900083E0089581E008952091D2013091D30131
:1018A0002617370748F06115710539F42091E800D3
:1018B0002E772093E80001C0B901FC0120E06115FA
:1018C000710591F18091CB01882309F440C08530E6
:1018D00009F43FC08091E80083FD3DC08091E8009D
:1018E00082FD2FC08091E80080FFE9CF2091F300B6
:1018F0008091F20090E0922B6115710559F08830CB
:10190000910540F424912093F100319661507109C2
:101910000196F2CF21E0089709F020E08091E800DD
:101920008E778093E800CBCF2111CCCF0AC0809175
:10193000CB01882361F0853061F08091E80083FD60
:101940000AC08091E80082FFF2CF80E0089582E033
:10195000089583E0089581E00895982F973058F511
:101960009093E900981739F07091EC002091ED0008
:101970005091F00003C0242F762F50E021FF19C0B2
:101980003091EB003E7F3093EB003091ED003D7FD6
:101990003093ED003091EB0031603093EB007093A9
:1019A000EC002093ED005093F0002091EE0027FF13
:1019B00007C09F5FD3CF8F708093E90081E00895C7
:1019C00080E008958091CC0187FF11C08091E800EC
:1019D00082FD05C08091CB018111F8CF11C08091AB
:1019E000E8008B770BC08091CB01882349F0809170
:1019F000E80080FFF8CF8091E8008E778093E800C0
:101A000008952091E4003091E50095E64091EC00C6
:101A1000842F817040FF22C08091E80080FD1CC0AF
:101A20008091CB01882391F0853091F08091EB007B
:101A300085FD10C04091E4005091E5004217530726
:101A400029F39A01915011F784E0089582E00895F6
:101A500083E0089581E0089580E008954091E800D2
:101A600042FFDECF08950E94A10D0E94A90DE0EE75
:101A7000F0E0808181608083E8EDF0E080818F7705
:101A8000808319BCA7EDB0E08C918E7F8C93808110
:101A90008F7E80831092CA0108950F931F93CF9376
:101AA000DF930E94A10D0E94A90DC8EDD0E08881AE
:101AB0008F77888388818068888388818F7D8883F9
:101AC00019BC1092CB011092C7011092C90110925B
:101AD000C80100EE10E0F80180818B7F808388814F
:101AE0008160888342E060E080E00E94AD0CE1EE1E
:101AF000F0E080818E7F8083E2EEF0E08081816083
:101B00008083808188608083F80180818E7F8083DC
:101B1000888180618883DF91CF911F910F91089513
:101B2000E8EDF0E080818F7E8083E7EDF0E080815A
:101B30008160808384E082BF81E08093CA010C943D
:101B40004D0DE8EDF0E080818E7F80831092E20001
:101B500008951092DA001092E10008951F920F92FA
:101B60000FB60F9211242F933F934F935F936F9370
:101B70007F938F939F93AF93BF93EF93FF93809146
:101B8000E10082FF0BC08091E20082FF07C08091DC
:101B9000E1008B7F8093E1000E94C3098091DA000D
:101BA00080FF1FC08091D80080FF1BC08091DA00A9
:101BB0008E7F8093DA008091D90080FF0DC080E194
:101BC00089BD82E189BD09B400FEFDCF81E080932B
:101BD000CB010E94A60905C019BC1092CB010E943E
:101BE000B8098091E10080FF19C08091E20080FF78
:101BF00015C08091E2008E7F8093E2008091E20028
:101C000080618093E2008091D80080628093D80048
:101C100019BC85E08093CB010E94CB0A8091E10042
:101C200084FF30C08091E20084FF2CC080E189BD38
:101C300082E189BD09B400FEFDCF8091D8008F7D7F
:101C40008093D8008091E1008F7E8093E1008091A5
:101C5000E2008F7E8093E2008091E20081608093B9
:101C6000E2008091C701882311F084E007C08091D1
:101C7000E30087FD02C081E001C083E08093CB01D7
:101C80000E942A0B8091E10083FF29C08091E2002D
:101C900083FF25C08091E100877F8093E10082E08F
:101CA0008093CB011092C7018091E1008E7F8093D9
:101CB000E1008091E2008E7F8093E2008091E2005B
:101CC00080618093E20042E060E080E00E94AD0C21
:101CD0008091F00088608093F0000E94BF09FF911E
:101CE000EF91BF91AF919F918F917F916F915F9194
:101CF0004F913F912F910F900FBE0F901F9018950D
:101D00001F920F920FB60F9211242F933F934F9370
:101D10005F936F937F938F939F93AF93BF93CF9373
:101D2000DF93EF93FF93C091E900CF708091EC00B7
:101D3000D82FD17080FDD0E81092E9008091F0009A
:101D4000877F8093F00078940E94C40E1092E9007F
:101D50008091F00088608093F000CD2BCF70C0930D
:101D6000E900FF91EF91DF91CF91BF91AF919F91EA
:101D70008F917F916F915F914F913F912F910F9034
:101D80000FBE0F901F9018951F93CF93DF93CDB781
:101D9000DEB7AA970FB6F894DEBF0FBECDBFECEC4E
:101DA000F1E088E08E0F9091F10091938E13FBCFBC
:101DB0000E94180A8091E80083FF1FC18091CC0126
:101DC0009091CD01492F50E04A30510508F015C1DE
:101DD000FA01EA5AFF4F0C94F124803881F08238DE
:101DE00009F00BC18091D0018F708093E900809140
:101DF000EB0085FB882780F91092E90006C08091EE
:101E0000C8019091C901911182609091E800977F7B
:101E10009093E8008093F1001092F100C8C0282F41
:101E20002D7F09F0EAC0882319F0823061F0E5C007
:101E30008091CE01813009F0E0C0933009F080E05C
:101E40008093C9012BC08091CE01811127C0809160
:101E5000D0018F7009F4D1C08093E9002091EB008C
:101E600020FF1CC0933021F48091EB00806214C0ED
:101E70009091EB0090619093EB0021E030E0A9019C
:101E800002C0440F551F8A95E2F74093EA00109272
:101E9000EA008091EB0088608093EB001092E900EB
:101EA0008091E800877F86C08111A7C01091CE0184
:101EB0001F778091E3008078812B8093E3008091ED
:101EC000E800877F8093E8000E94E20C8091E800A0
:101ED00080FFFCCF8091E30080688093E3001111C4
:101EE00002C082E001C083E08093CB0186C08058AD
:101EF000823008F082C08091CE019091CF018C3D5C
:101F000053E0950779F583E08A838AE289834FB7A6
:101F1000F894DE01139620E03EE051E2E32FF0E07A
:101F200050935700E49120FF03C0E295EF703F5FAC
:101F3000EF708E2F90E0EA3010F0C79601C0C09687
:101F40008D939D932F5F243149F74FBF8091E80017
:101F5000877F8093E8006AE270E0CE0101960E94DC
:101F6000E90B14C0AE014F5F5F4F6091D0010E943A
:101F7000300BBC01892B09F440C09091E800977F99
:101F80009093E80089819A810E944C0C8091E8002E
:101F90008B778093E80031C0803879F58091E80034
:101FA000877F8093E8008091C7018093F100809142
:101FB000E8008E778093E8000E94E20C1EC0811139
:101FC0001CC09091CE019230C0F48091E800877FD0
:101FD0008093E8009093C7010E94E20C8091C701B2
:101FE000811106C08091E30087FD02C081E001C03D
:101FF00084E08093CB010E94040A8091E80083FF73
:102000000AC08091E800877F8093E8008091EB0010
:1020100080628093EB00AA960FB6F894DEBF0FBEE5
:10202000CDBFDF91CF911F91089590935B01809375
:102030005A010895E0915A01F0915B01309721F027
:102040000190F081E02D099480E00895EF92FF92D5
:102050000F931F93CF93DF93E0915A01F0915B01AF
:102060003097B1F18C010280F381E02D09958091C8
:10207000B60182FF2DC080FF04C088EB93E00E9470
:102080004A05E80118E082EBE82E83E0F82E809103
:10209000B60180FF0BC088811F928F93FF92EF9251
:1020A0000E94E3050F900F900F900F901150219612
:1020B0001111EDCF8091B60180FF0AC080EB93E053
:1020C000DF91CF911F910F91FF90EF900C944A05F3
:1020D000DF91CF911F910F91FF90EF900895E091C4
:1020E0005A01F0915B01309721F00480F581E02DD9
:1020F000099408952091580130915901821793074E
:1021000071F09093590180935801E0915A01F09138
:102110005B01309721F00680F781E02D0994089546
:1021200020915601309157018217930771F09093D7
:10213000570180935601E0915A01F0915B0130976D
:1021400021F00084F185E02D0994089508950C9400
:10215000A6100E94531C0C94EC05CF92DF92EF92D4
:10216000FF920F931F93CF93DF9300D000D000D046
:10217000CDB7DEB70E9409068DE5C82E81E0D82EC6
:1021800000E010E0E02E802F0E945B06F6014191F6
:102190006F01F42EF826B1F40F5F1F4F0E301105BA
:1021A00089F78FEF89838A831B820E945C1C816080
:1021B000782F9D838C8349815A816B818D810E9408
:1021C0006C1147C09091B60191FF04C08E830E94AC
:1021D00064068E8120E030E04F2D50E0922FBA014E
:1021E000022E02C0759567950A94E2F760FF2BC036
:1021F0002983EA8221E030E0690102C0CC0CDD1CB9
:102200009A95E2F790E08C219D21892B09F420E03A
:102210002B830E945C1C8160782F9D838C83498175
:102220005A816B818D810E946C1149815A816B8129
:102230007C818D810E94D61BF801E35AFE4F80817C
:10224000C826C08206C02F5F3F4F2830310531F6C7
:10225000A3CF0E94D51B0E941D1F10915C010E94FC
:102260001A10181741F10E941A1080935C01909186
:10227000B60192FF0EC090FF0CC01F928F938AECA4
:1022800093E09F938F930E94E3050F900F900F9020
:102290000F9080915C0126960FB6F894DEBF0FBEBA
:1022A000CDBFDF91CF911F910F91FF90EF90DF9005
:1022B000CF900C94E71B26960FB6F894DEBF0FBEA6
:1022C000CDBFDF91CF911F910F91FF90EF90DF90E5
:1022D000CF9008950C94A606CF93DF93CDB7DEB7C9
:1022E0002B970FB6F894DEBF0FBECDBF942F4F8350
:1022F000252F588769877A878B874A855B85452B89
:1023000021F02F3F09F59F3FF9F4DE01119686E099
:10231000FD0111928A95E9F785E0FE01379601905B
:102320000D928A95E1F749815A816B817C818D817B
:102330009E810E9490182B960FB6F894DEBF0FBEB8
:10234000CDBFDF91CF9108954F81588569857A85FA
:102350008B850E94D61BD9CFCF93882309F4CDC09B
:10236000C82F823859F40E941A1081FDC6C089E333
:102370000E941B1B0E94941B89E30CC0833879F4D4
:102380000E941A1080FDB9C083E50E941B1B0E94A9
:10239000941B83E50E94381BCF910C94941B8438C6
:1023A00059F40E941A1082FDA8C087E40E941B1BEA
:1023B0000E94941B87E4EECF8CEF8C0F813A48F497
:1023C0008C2F0E944722811198C08C2F0E941B1BCA
:1023D000E3CF80E28C0F883048F4C77081E001C001
:1023E000880FCA95EAF70E945A1BD6CF8BE58C0F4F
:1023F000833078F4C53A29F0C63A31F083E890E0AA
:1024000005C081E890E002C082E890E0CF910C9492
:102410007A1088E58C0F853108F06FC0C83A61F1F9
:10242000C93A69F1CA3A71F1CB3A79F1CC3A81F102
:10243000CD3A89F1CE3A91F1CF3A99F1C13BA1F170
:10244000C03BA9F1C23BB1F1C33BB9F1C43BC1F1FF
:10245000C53BC9F1C63BD1F1C73BD9F1C83BE1F15E
:10246000C93BE9F1CA3BF1F1CB3BF9F1CC3B09F4B3
:102470003FC080E090E03EC082EE90E03BC089EE3D
:1024800090E038C08AEE90E035C085EB90E032C035
:1024900086EB90E02FC083EB90E02CC084EB90E0C3
:1024A00029C087EB90E026C08CEC90E023C08DEC37
:1024B00090E020C083E891E01DC08AE891E01AC056
:1024C00082E991E017C084E991E014C081E292E0D2
:1024D00011C083E292E00EC084E292E00BC085E27C
:1024E00092E008C086E292E005C087E292E002C076
:1024F0008AE292E0CF910C949010CF9108958823B6
:1025000009F44BC0823859F40E941A1081FF45C06B
:1025100089E30E941B1B0E94941B89E30CC0833833
:1025200071F40E941A1080FF38C083E50E941B1BC3
:102530000E94941B83E50E94381B0C94941B8438E2
:1025400059F40E941A1082FF28C087E40E941B1BC6
:102550000E94941B87E4EFCF9CEF980F913A58F3B9
:1025600090E2980F983050F4877091E001C0990F75
:102570008A95EAF7892F0E94601BDFCF9BE5980FB1
:10258000933020F480E090E00C947A10885A8531E2
:1025900020F480E090E00C9490100895882321F0BE
:1025A0000E945A1B0C94941B0895882321F00E94CA
:1025B000601B0C94941B0895CF92DF92EF92FF92D0
:1025C0000F931F93CF93DF9300D000D000D0CDB7EF
:1025D000DEB725E0FC01DE01119601900D922A95EF
:1025E000E1F7FC0140813181F280258122952F7035
:1025F00063817481672B09F4D8C23F3F19F44F3FC0
:1026000009F4D3C26C0149833A8389819A812E836C
:102610000E94DA1A182F092F0E94D91A0E94E9196C
:10262000E02FE295EF70F0E0E05AFF4F2E810C941E
:10263000F124802F807F902F9F70092F882311F025
:102640000295007FFF2049F0002309F45FC2802F2C
:102650000E946D1B0E94941B59C2812F0E947F1201
:10266000002309F4A2C2802F0E94731B26960FB686
:10267000F894DEBF0FBECDBFDF91CF911F910F91B8
:10268000FF90EF90DF90CF900C94941B802F807F71
:10269000902F9F70092F803211F00295007F112337
:1026A00019F0113001F129C0FF20A9F0802F222359
:1026B00049F1213039F526960FB6F894DEBF0FBEEA
:1026C000CDBFDF91CF911F910F91FF90EF90DF90E1
:1026D000CF900C947D1B222319F0213009F465C2A0
:1026E0000E94801B2CC0FF20E9F0263008F05DC25C
:1026F0000E94571B802329F022C0FF20F1F02111F6
:1027000015C0802F26960FB6F894DEBF0FBECDBF42
:10271000DF91CF911F910F91FF90EF90DF90CF90BD
:102720000C94CE12253008F040C209C0F601858114
:1027300080FFECC18F708583E4CF2111FBC1802F16
:1027400069C1202F26952695237030E0211531058B
:1027500021F021303105C9F028C2FF2021F0812F5E
:10276000902F937002C080E090E026960FB6F89408
:10277000DEBF0FBECDBFDF91CF911F910F91FF90B4
:10278000EF90DF90CF900C947A10FF2021F0812FF2
:10279000902F937002C080E090E026960FB6F894D8
:1027A000DEBF0FBECDBFDF91CF911F910F91FF9084
:1027B000EF90DF90CF900C949010812FFF2019F0B4
:1027C0000E94A31D02C00E940B1E26960FB6F8940D
:1027D000DEBF0FBECDBFDF91CF911F910F91FF9054
:1027E000EF90DF90CF900C94901E802F837009F0B3
:1027F00078C0F110DAC1812F829586958770880F95
:10280000880F912F9F70C92ED12CE12CF12C082E0E
:1028100004C0CC0CDD1CEE1CFF1C0A94D2F714FF84
:1028200012C04FE050E060E070E004C0440F551F5C
:10283000661F771F8A95D2F7CB01BA016095709514
:102840008095909503C060E070E0CB01202F269525
:1028500026952370422F50E042305105D1F043308D
:10286000510559F16C297D298E299F294130510547
:1028700041F126960FB6F894DEBF0FBECDBFDF91B3
:10288000CF911F910F91FF90EF90DF90CF900C941C
:10289000FE196C297D298E299F2926960FB6F8945A
:1028A000DEBF0FBECDBFDF91CF911F910F91FF9083
:1028B000EF90DF90CF900C94101A0E94FE19C70180
:1028C000B60126960FB6F894DEBF0FBECDBFDF91DE
:1028D000CF911F910F91FF90EF90DF90CF900C94CC
:1028E000EC19FF2019F0802F817001C08695882394
:1028F00009F45BC1812F829586958770880F880FB8
:10290000912F9F70C92ED12CE12CF12C082E04C0E0
:10291000CC0CDD1CEE1CFF1C0A94D2F714FF12C075
:102920004FE050E060E070E004C0440F551F661FA8
:10293000771F8A95D2F7CB01BA0160957095809583
:10294000909503C060E070E0CB01202F269526957E
:102950002370422F50E042305105D1F043305105F1
:1029600059F16C297D298E299F294130510541F16A
:1029700026960FB6F894DEBF0FBECDBFDF91CF9184
:102980001F910F91FF90EF90DF90CF900C94B51AAC
:102990006C297D298E299F2926960FB6F894DEBFD3
:1029A0000FBECDBFDF91CF911F910F91FF90EF90A0
:1029B000DF90CF900C94C71A0E94B51AC701B601D8
:1029C00026960FB6F894DEBF0FBECDBFDF91CF9134
:1029D0001F910F91FF90EF90DF90CF900C94A31A6E
:1029E000103F41F118F4103E48F48BC0123F09F437
:1029F00050C0D8F1133F09F460C083C01F70802F0E
:102A00008F71FF2021F00E943C1A812F7BCE0E9403
:102A10005D1A812F26960FB6F894DEBF0FBECDBF8C
:102A2000DF91CF911F910F91FF90EF90DF90CF90AA
:102A30000C94D512FF20A9F0253008F0B6C0802FE5
:102A40008F7126960FB6F894DEBF0FBECDBFDF9113
:102A5000CF911F910F91FF90EF90DF90CF900C944A
:102A6000821A263008F0A1C0EACFFF20A1F0802F03
:102A70008F7126960FB6F894DEBF0FBECDBFDF91E3
:102A8000CF911F910F91FF90EF90DF90CF900C941A
:102A90003C1AFF2061F3802F8F7126960FB6F894B1
:102AA000DEBF0FBECDBFDF91CF911F910F91FF9081
:102AB000EF90DF90CF900C945D1AFF2091F0802F63
:102AC0008F7126960FB6F894DEBF0FBECDBFDF9193
:102AD000CF911F910F91FF90EF90DF90CF900C94CA
:102AE000271A26960FB6F894DEBF0FBECDBFDF9132
:102AF000CF911F910F91FF90EF90DF90CF900C94AA
:102B0000221AFF20A1F0222309F4B1CF812F2696AB
:102B10000FB6F894DEBF0FBECDBFDF91CF911F91EE
:102B20000F91FF90EF90DF90CF900C94AC11222387
:102B300009F4B1CF812F26960FB6F894DEBF0FBEF1
:102B4000CDBFDF91CF911F910F91FF90EF90DF905C
:102B5000CF900C947F12402F4F70612FC6010E94BE
:102B60001D1D26960FB6F894DEBF0FBECDBFDF91B8
:102B7000CF911F910F91FF90EF90DF90CF900C9429
:102B80003419402F4F70612FC60126960FB6F89466
:102B9000DEBF0FBECDBFDF91CF911F910F91FF9090
:102BA000EF90DF90CF900C94201D26960FB6F894EE
:102BB000DEBF0FBECDBFDF91CF911F910F91FF9070
:102BC000EF90DF90CF9008950E947A1B0E94491BDE
:102BD0000E94941B0E94C21F0E94901E80E090E001
:102BE0000E947A1080E090E00C9490100E946A1B82
:102BF0000C94E4150E94DA1A292F22952F7030E0E8
:102C00002C3031054CF42A3031056CF42250310956
:102C10002230310588F407C02C30310549F02F30BF
:102C2000310531F009C0803E48F0803F29F406C0EC
:102C300093FB882780F9089580E0089581E0089546
:102C4000CF93DF9300D000D01F92CDB7DEB70F90A7
:102C50000F900F900F900F90DF91CF910895CF9329
:102C6000DF9300D000D000D0CDB7DEB726960FB6E8
:102C7000F894DEBF0FBECDBFDF91CF9108951F93B3
:102C8000CF93DF93C0916B0116E080916C01C81760
:102C900099F0D0E01C9FF0011D9FF00D1124E35925
:102CA000FE4F4081518162817381848195810E94B0
:102CB0002F162196C770E9CFDF91CF911F9108950C
:102CC00040919D0150919E0160919F017091A001E2
:102CD0008091A1019091A2010C942F168091A201E4
:102CE00082958F7009F054C080919F01882309F468
:102CF0004FC080916B01A0916C0160919D0170911A
:102D00009E014091A0015091A101B6E08A1709F4FB
:102D10003FC090E041155105C1F17F3F11F46F3F75
:102D2000A1F1B89FF001B99FF00D1124E359FE4FB6
:102D3000218172132AC02081621327C022812111B0
:102D400024C0238134812417350710F42150310920
:102D5000241B350B283C3105C0F42091A2012F70B3
:102D600020612093A20126E0289FF001299FF00D09
:102D70001124EE58FE4F80818F70806180838DE931
:102D800091E00E94DC120C943F1601968770BECF32
:102D90000895CF92DF92EF92FF920F931F93CF93FC
:102DA000DF93CDB7DEB762970FB6F894DEBF0FBEE4
:102DB000CDBF8C0185E0F801DE011D9601900D92DA
:102DC0008A95E1F7D8014C9111965C911197129672
:102DD0006C9112971396CD90DC90149730919D01D1
:102DE00070919E018091A0019091A101009709F43A
:102DF0006BC17F3F19F43F3F09F466C1E0909F012A
:102E0000EE2009F4C0C02091A201C816D90628F00E
:102E1000F601E81BF90BCF0104C0809590958C0D4D
:102E20009D1DFF24F394883C910578F0F12C207FC0
:102E300009F0C6C07C2DD98AC88A89890E942016CB
:102E40008DE991E00E94DC12B1C0822F807F09F0F1
:102E500046C0751314C0341312C0611110C02F7016
:102E600020612093A2010E9460168DE991E00E94EA
:102E7000DC128091A201D80115968C932EC0CD282A
:102E800019F15F3F11F44F3FF9F0F62E61111CC0AC
:102E900080916B0120916C0136E0821709F45AC0D1
:102EA00090E0389FF001399FF00D1124E359FE4F57
:102EB0007181571306C07081471303C0728171116D
:102EC00003C001968770E9CFF62E662309F418C176
:102ED0008091A20181608093A201F12C11C1751330
:102EE00008C0341306C0611104C08091A201D8014A
:102EF000C3C04D875E878D859E856A8B0E94FA15BB
:102F00006A898823E1F16623D1F12091A201822F01
:102F100082958F7090E0029774F080919D0190915E
:102F20009E0198878F831986DB86CA862C87CE01FF
:102F300007960E94DC1286E0F801ADE9B1E001904D
:102F40000D928A95E1F70E946E160E946016FF248A
:102F5000F394D6C04D875E878D859E850E94DA1AD0
:102F6000292F22952F7030E0223031050CF0BCC0A3
:102F70009F7009F0B6C0805E883008F4C1C0C801F7
:102F80000E94DC12E4CFC816D90608F453C0F6013B
:102F9000E81BF90BCF01883C910508F450C0F12CD7
:102FA0007C2DD98AC88A89890E942016EDE9F1E032
:102FB00086E0DF011D928A95E9F70E946016A0C0A5
:102FC000751314C0341312C0611110C08091A20196
:102FD000F8018583C8010E94DC1286E0EDE9F1E08A
:102FE000DF011D928A95E9F7FE2C8AC04D875E8726
:102FF0008D859E856A8B0E94FA156A89882309F45B
:10300000BECF662309F4BBCF2091A201822F829507
:103010008F7090E002970CF48ECF80919D0190917B
:103020009E019A8389831B82DD82CC822E83CE010E
:1030300001967FCF809590958C0D9D1DACCFF62E7F
:10304000662309F49CCF75132EC034132CC0209135
:10305000A20120FD1FC0822F82958F70D9F0D80168
:1030600015962C9315978F3049F08F5F982F929576
:10307000907F822F8F70892B15968C93C8010E94A8
:10308000DC1286E0F801ADE9B1E001900D928A957D
:10309000E1F793CF86E0F801ADE9B1E001900D9240
:1030A0008A95E1F72DC04D875E878D859E850E94AC
:1030B000FA15811140CF8091A20181608093A20115
:1030C000C8010E94DC121CC0662309F458CF4D874A
:1030D0005E878D859E850E94FA15882309F44FCF5F
:1030E0002ACF811148CF0CC0243031050CF047CFD6
:1030F0009F7009F440CFF8019581907F09F03BCF94
:103100008F2D62960FB6F894DEBF0FBECDBFDF9154
:10311000CF911F910F91FF90EF90DF90CF90089586
:103120001F93CF93DF93CDB7DEB72C970FB6F894EC
:10313000DEBF0FBECDBF4F83588769877A878B87E5
:103140009C87CE0107960E94C916882369F08F815B
:1031500098852A853B85232BF1F19F3F09F063C0B9
:103160008F3F09F060C037C086E0FE013796DE0170
:10317000119601900D928A95E1F76F817885EA8525
:10318000FB85309741F17F3F11F46F3F21F1209192
:103190006C0130E0C90101968770992740916B015D
:1031A00050E08417950709F447C069837A83FD834B
:1031B000EC8396E0929FD001939FB00D1124A35908
:1031C000BE4FFE01319601900D929A95E1F78093E2
:1031D0006C010E943F1616E080916B0190916C018A
:1031E0008917C1F1189FC001112483599E4F0E9475
:1031F000C916882379F1E0916B011E9FF00111241B
:10320000E359FE4F408151816281738184819581B0
:103210000E942F1680916B0190E00196877099278C
:1032200080936B01D9CF4F81588569857A858B85CD
:103230009C850E942F16CFCF0E94F61510926C012C
:1032400010926B01EDE9F1E086E0DF011D928A95B5
:10325000E9F7C1CF2C960FB6F894DEBF0FBECDBFF5
:10326000DF91CF911F910895DF92EF92FF920F931C
:103270001F93CF93DF93FC01892B09F48AC0E12CC3
:10328000F12CDD24D394EF0121968491853709F444
:1032900061C058F4843708F04EC0843008F06AC02A
:1032A0008130D1F0823071F174C0883709F45DC08B
:1032B00050F4863709F455C0873709F06AC08E2D5F
:1032C0000E94671B54C09CE7980F903708F061C0BC
:1032D0008F770E947F1250C08F010E5F1F4FFE013B
:1032E000849190E2980F983050F48770FD2D01C0C2
:1032F000FF0F8A95EAF78F2F0E946D1B14C00E9462
:10330000AC1113C08F010E5F1F4FFE01C49180E20C
:103310008C0F883060F4C7708D2D01C0880FCA955E
:10332000EAF70E94731B0E94941BE80125C08C2FB2
:103330000E947F12FACF9F012E5F3F4FFE01C49182
:10334000CC2369F08FE99FE00197F1F700C00000FE
:10335000C150F6CF9F012E5F3F4FFE01F490E9016F
:103360000BC00E94571BE82E07C00E946A1B0E94D8
:10337000941B02C00E94AC118F2D882341F0EFE90D
:10338000FFE03197F1F700C000008150F6CFFE0159
:103390007ACFDF91CF911F910F91FF90EF90DF9047
:1033A00008956093A7017093A8018093A901909359
:1033B000AA010E94E51B0C94E4156093A30170938D
:1033C000A4018093A5019093A6010E94E61B0C9492
:1033D000E41508950C94D1190F931F930091A70140
:1033E0001091A8012091A9013091AA01602B712BA5
:1033F000822B932B1F910F910C94D1190F931F9334
:103400000091A7011091A8012091A9013091AA0172
:1034100060237123822393231F910F910C94D11960
:103420000F931F930091A7011091A8012091A9016A
:103430003091AA0160277127822793271F910F914E
:103440000C94D11960E070E0CB010C94DD190F935E
:103450001F9341E050E060E070E08A019B0104C0EE
:10346000000F111F221F331F8A95D2F7C901B8011F
:103470001F910F910C94DD190F931F9341E050E0C1
:1034800060E070E004C0440F551F661F771F8A95E7
:10349000D2F78091A3019091A401A091A501B091D0
:1034A000A6018A019B01082B192B2A2B3B2BC90152
:1034B000B8011F910F910C94DD190F931F9341E0F8
:1034C00050E060E070E004C0440F551F661F771F96
:1034D0008A95D2F740955095609570958091A3019B
:1034E0009091A401A091A501B091A6018A019B0130
:1034F000082319232A233B23C901B8011F910F91E7
:103500000C94DD190F931F9341E050E060E070E0F0
:1035100004C0440F551F661F771F8A95D2F780910C
:10352000A3019091A401A091A501B091A6018A01E7
:103530009B01082719272A273B27C901B8011F919A
:103540000F910C94DD190F931F930091A30110911B
:10355000A4012091A5013091A601602B712B822B33
:10356000932B1F910F910C94DD190F931F930091D2
:10357000A3011091A4012091A5013091A60160231F
:103580007123822393231F910F910C94DD190F93C4
:103590001F930091A3011091A4012091A5013091E6
:1035A000A60160277127822793271F910F910C9402
:1035B000DD190895CF92DF92EF92FF920F931F9340
:1035C000CF93DF938C01C090A701D090A801E09029
:1035D000A901F090AA014091A3015091A40160912A
:1035E000A5017091A601C42AD52AE62AF72ACFE1BF
:1035F000D0E0D701C6010C2E04C0B695A7959795CB
:1036000087950A94D2F780FF07C0B8018C2F0E94DB
:10361000F31C8130910531F4219758F7B80180E00F
:103620000E94F31CDF91CF911F910F91FF90EF90BB
:10363000DF90CF90089520910B0130910C01F9019A
:1036400032969FEF40E05191581789F09F3F19F44F
:10365000511101C0942F4F5F4630A9F79F3F39F0B9
:10366000F901E90FF11D97FDFA95828308950895F8
:1036700020910B0130910C01F9013296285F3F4FE8
:103680009081981301C010823196E217F307C1F7B9
:10369000089581E090E0E0910B01F0910C01E80FBA
:1036A000F91F1082019688309105A9F7089580913D
:1036B000B50108959091B501892B8093B5010895C6
:1036C00080959091B50189238093B50108958093E9
:1036D000B50108951092B50108959091B401892B18
:1036E0008093B401089580959091B40189238093CB
:1036F000B40108951092B40108958093AB01089528
:103700001092AB01089580910B0190910C01FC0186
:1037100031969C01285F3F4F80E0919191118F5F1E
:10372000E217F307D1F70895E0910B01F0910C0136
:103730008091B5018083E0910B01F0910C019081A3
:103740008091B401892B80838091AB01882361F043
:10375000E0910B01F0910C019081892B80830E94F4
:10376000831B81111092AB0180910B0190910C0190
:103770000C94261090933301809332010895829522
:10378000982F9C7C392F36953695282F237344E04B
:10379000249FC0011124932F982B292F2A7A269534
:1037A000892F8575880F822B08950895CF93DF9315
:1037B00000D000D01F92CDB7DEB70F900F900F90C2
:1037C0000F900F90DF91CF910895089508950C9474
:1037D0006A118091CB01843021F11092B70120E46D
:1037E00088E190E00FB6F894A895809360000FBE32
:1037F0002093600083B7817F846083BF83B781603B
:1038000083BF7894889583B78E7F83BF0FB6F89473
:10381000A89580916000886180936000109260009C
:103820000FBE089508950895CF930E94121C0E9420
:1038300009060E94131CC0E08C2F0E945B068111B8
:1038400004C0CF5FCE30C1F701C081E0CF910895B1
:103850000C94F6151F920F920FB60F9211248F93AE
:103860009F93AF93BF938091B701811113C0809153
:10387000B8019091B901A091BA01B091BB014196F4
:10388000A11DB11D8093B8019093B901A093BA0115
:10389000B093BB01BF91AF919F918F910F900FBEDD
:1038A0000F901F90189582E084BD93E095BD9AEF2C
:1038B00097BD80936E0008952FB7F8948091B8015A
:1038C0009091B901A091BA01B091BB012FBF0895A9
:1038D0002FB7F8946091B8017091B9018091BA0145
:1038E0009091BB012FBF0895CF92DF92EF92FF928C
:1038F0000F931F932FB7F8944091B8015091B901DD
:103900006091BA017091BB012FBF6A017B01EE2467
:10391000FF248C0120E030E0C016D106E206F30659
:1039200010F4415051099A01281B390BC9011F910C
:103930000F91FF90EF90DF90CF9008951F920F921C
:103940000FB60F9211248F939F93AF93BF938091E3
:10395000B8019091B901A091BA01B091BB01019653
:10396000A11DB11D8093B8019093B901A093BA0134
:10397000B093BB01BF91AF919F918F910F900FBEFC
:103980000F901F9018950E94330DF8942FEF87EA3F
:1039900091E6215080409040E1F700C0000087E0B0
:1039A00090EBDC018093D4019093D501A093D601D4
:1039B000B093D7019CE088E10FB6F894A895809366
:1039C00060000FBE90936000FFCF28E0929FF0014F
:1039D0001124E80FF11DE052FF4F9491892F8F7051
:1039E00092959F700895CF93C82FCB010E94E51C3C
:1039F000282F30E080E1989FA0011124422B532B07
:103A00004038510519F480E090E015C09770E92F17
:103A1000F0E088E0C89FE00DF11D112484E0EE0F76
:103A2000FF1F8A95E1F7E20FF31FEE0FFF1FE05033
:103A3000F84985919491CF91089580E090E00895A0
:103A400008958091BE0180FF0BC06091100185E058
:103A5000689FB001112475956795759567952BC082
:103A600081FF09C06091100185E0689FB0011124B9
:103A70007595679520C082FF07C06091100185E0B1
:103A8000689FB001112417C09091BF019923D1F014
:103A900060910F01961788F72091100185E0289F0B
:103AA00090011124929FA001939F500D112470E06A
:103AB000CA010E94DD246038710540F4611571056A
:103AC00039F002C065E070E0862F08958FE7089511
:103AD00081E008958091BE0180FF08C060910E01D1
:103AE00070E0759567957595679521C081FF06C053
:103AF00060910E0170E07595679519C082FF04C052
:103B000060910E0170E010C09091BF019923C1F047
:103B100060910D019617A0F780910E01899FC00159
:103B2000112470E00E94DD246038710528F46115CD
:103B3000710521F0862F08958FE7089581E008959B
:103B400061E070E0F4CF803F21F40E94211D819557
:103B500004C0813F29F40E94211D8093C201089571
:103B6000823F21F40E94211D819504C0833F29F4E6
:103B70000E94211D8093C1010895893F19F40E947C
:103B80006A1D05C08A3F31F40E946A1D81958093A9
:103B9000C30108958B3F21F40E946A1D819504C0E2
:103BA0008C3F29F40E946A1D8093C4010895843FCC
:103BB00021F48091C001816017C0853F21F480917C
:103BC000C001826011C0863F21F48091C0018460F1
:103BD0000BC0873F21F48091C001886005C0883FF9
:103BE00031F48091C00180618093C00108958D3FC0
:103BF00021F48091BE0181600BC08E3F21F4809141
:103C0000BE01826005C08F3F29F48091BE018460AF
:103C10008093BE010895803F39F48091C20187FFEF
:103C20006CC01092C20169C0813F29F48091C20129
:103C30001816BCF362C09091C101823F29F497FF2E
:103C40005CC01092C10159C0833F19F41916CCF31E
:103C500054C0893F41F48091C30118160CF04DC047
:103C60001092C3014AC08A3F29F48091C30187FFA3
:103C700044C0F6CF8B3F39F48091C40187FF3DC02B
:103C80001092C4013AC08C3F29F48091C4011816E7
:103C9000BCF333C0843F21F48091C0018E7F17C0F4
:103CA000853F21F48091C0018D7F11C0863F21F4B2
:103CB0008091C0018B7F0BC0873F21F48091C001B0
:103CC000877F05C0883F31F48091C0018F7E80934B
:103CD000C00113C08D3F21F48091BE018E7F0BC0C7
:103CE0008E3F21F48091BE018D7F05C08F3F29F466
:103CF0008091BE018B7F8093BE018091C1018111B3
:103D00000EC08091C20181110AC08091C30181114E
:103D100006C08091C401811102C01092BF010895B4
:103D20008091B60183FF7EC08CEF93E00E944A052C
:103D30008091C0011F928F9387EF93E09F938F93A1
:103D40000E94E30585EF93E00E944A058091C1013E
:103D5000282F082E000C330B3F938F9382EF93E0B4
:103D60009F938F930E94E30580EF93E00E944A05A2
:103D70008091C201282F082E000C330B3F938F93A4
:103D80008DEE93E09F938F930E94E3058BEE93E07B
:103D90000E944A058091C301282F082E000C330B86
:103DA0003F938F9388EE93E09F938F930E94E30558
:103DB00086EE93E00E944A058091C401282F082EC8
:103DC000000C330B3F938F9383EE93E09F938F937D
:103DD0000E94E30580EE93E00E944A058091BF01B6
:103DE0001F928F938DED93E09F938F930E94E30535
:103DF0008BED93E00E944A058091BE011F928F9344
:103E000088ED93E09F938F930E94E30585ED93E007
:103E10000E944A058DB79EB74C960FB6F8949EBF88
:103E20000FBE8DBF80EC91E00E946F100E945C1C61
:103E30009093BD018093BC0108951F93CF93DF93AE
:103E40008091BC019091BD010E94741CAC019091C5
:103E5000BF01992321F02091110130E006C020918B
:103E600012018AE0289F900111244217530708F499
:103E700085C08091C101C091C201D091C301109150
:103E8000C401811107C0C11175C0D11173C01111D6
:103E900071C074C09F3F19F09F5F9093BF011816C7
:103EA00024F40E94211D8093C1018091C10187FFEC
:103EB00005C00E94211D81958093C1011C1624F428
:103EC0000E94211D8093C2018091C20187FF05C01D
:103ED0000E94211D81958093C2016091C1016623DA
:103EE00031F1C091C201CC2311F1062E000C770BE9
:103EF000880B990B0E94D82323E333E343E35FE36A
:103F00000E943C240E94A0236093C1016C2FCC0F1F
:103F1000770B880B990B0E94D82323E333E343E309
:103F20005FE30E943C240E94A0236093C2011D16FF
:103F300024F40E946A1D8093C3018091C30187FF0E
:103F400005C00E946A1D81958093C301111624F457
:103F50000E946A1D8093C4018091C40187FF05C03F
:103F60000E946A1D81958093C401DF91CF911F91BA
:103F70000C94901E9F3F09F08FCF97CFDF91CF9188
:103F80001F910895E0ECF1E085E0DF011D928A9534
:103F9000E9F71092BF011092BE0108958FE196E0FB
:103FA0000E944A051F9281E08F931F9285E08F93B4
:103FB00081ED95E09F938F930E94E3050F900F9002
:103FC0000F900F900F900F9008958330E9F128F42F
:103FD000813061F0823009F10895853009F462C0C2
:103FE00008F449C0863009F474C008958091120124
:103FF000262F30E0280F311D2F3F310524F4680FA4
:104000006093120103C08FEF80931201809112011F
:104010001F928F938AE095E072C080911101262F44
:1040200030E0280F311D2F3F310524F4680F6093D5
:10403000110103C08FEF80931101809111011F9234
:104040008F9388EF94E05BC080911001262F30E0C1
:10405000280F311D2F3F310524F4680F60931001A4
:1040600003C08FEF80931001809110011F928F93F6
:1040700085EE94E044C080910F01262F30E0280F98
:10408000311D2F3F310524F4680F60930F0103C0E9
:104090008FEF80930F0180910F011F928F9380ED1E
:1040A00094E02DC080910E01262F30E0280F311DA5
:1040B0002F3F310524F4680F60930E0103C08FEF8A
:1040C00080930E0180910E011F928F9387EB94E0F5
:1040D00016C080910D01262F30E0280F311D2F3F93
:1040E000310524F4680F60930D0103C08FEF8093B6
:1040F0000D0180910D011F928F938CE994E09F93A5
:104100008F930E94E3050F900F900F900F900895EA
:10411000833081F128F4813059F08230D1F0089554
:10412000853009F449C0B8F1863009F456C00895C5
:1041300080911201681720F4861B8093120102C03F
:1041400010921201809112011F928F938DE894E0DA
:1041500054C080911101681720F4861B80931101CF
:1041600002C010921101809111011F928F938BE771
:1041700094E043C080911001681720F4861B80935F
:10418000100102C010921001809110011F928F93B4
:1041900088E694E032C080910F01681720F4861BF6
:1041A00080930F0102C010920F0180910F011F92A6
:1041B0008F9383E594E021C080910E01681720F46D
:1041C000861B80930E0102C010920E0180910E0199
:1041D0001F928F938AE394E010C080910D016817BD
:1041E00020F4861B80930D0102C010920D01809176
:1041F0000D011F928F938FE194E09F938F930E9404
:10420000E3050F900F900F900F900895CF93C82F54
:104210001F928F9384E297E09F938F930E94E30510
:1042200081E090E0A0E0B0E0BC01CD0104C0660FE9
:10423000771F881F991FCA95D2F70E94EA190F901D
:104240000F900F900F90CF910C94F615CF9387326B
:1042500088F58E3108F00BC18E3009F487C0D8F490
:10426000873009F460C08B3009F44FC0863009F004
:1042700002C18091B601817F8E7F8093B60189E271
:1042800097E00E944A0586EE99E00E944A0581E087
:104290008093C60146C0863109F4B0C020F4803155
:1042A00009F47AC0E8C0893109F491C08B3109F46E
:1042B00049C0E1C0883349F150F4893209F4D5C0CE
:1042C000853309F4D2C0873209F0D5C0CEC083341B
:1042D00009F4CBC028F48A3308F4CDC08953C8C090
:1042E000883409F0C8C00E94F61585ED99E00E9457
:1042F0004A052FEF83ED90E3215080409040E1F795
:1043000000C000000E94C31C0CC080E597E041C0C3
:104310008CEB99E00E944A058091B6018160809300
:10432000B601C1E0ADC08091B601C82FC17080FF59
:10433000EFCF88EC99E00E944A058091B601817F19
:104340008E7F3FC09091B60191FBCC27C0F981E0F0
:10435000C827892FC0FB81F98093B601CC2319F0BF
:104360008FEA99E029C081EA99E013C09091B601E3
:1043700092FBCC27C0F981E0C827892FC0FB82F9C6
:104380008093B601CC2319F082E999E015C082E848
:1043900099E00E944A05C5CF9091B60193FBCC27C6
:1043A000C0F981E0C827892FC0FB83F98093B6014B
:1043B000CC2351F086E799E00E944A058091B6012E
:1043C00081608093B6015CC089E699E0E2CF8AE51E
:1043D00099E00E944A0585E399E00E944A058EEE25
:1043E00098E00E944A0581EC98E00E944A058CE71B
:1043F00098E00E944A058EE498E0CBCF80E498E0F4
:104400000E944A050E941A101F928F9386E298E03C
:104410009F938F930E94E30580910A011F928F93CF
:104420008FE098E09F938F930E94E3058091550160
:104430001F928F938CEF97E09F938F930E94E305D9
:104440000E94681C9F938F937F936F9385EE97E0F4
:104450009F938F930E94E3058DB79EB742960FB648
:10446000F8949EBF0FBE8DBF5CCF80E001C08D5120
:104470000E94062156CF83EE97E00E944A05C0E0D5
:104480008C2FCF91089580E0089580E00895CF9318
:10449000C82F8091C601813081F020F0823009F46C
:1044A0004FC046C1E0910B01F0910C0180818E302C
:1044B00069F0873009F03EC109C0E0910B01F0912D
:1044C0000C0180818E3011F0873061F48C2F0E94B6
:1044D0004322811104C08C2F0E9426212FC081E02D
:1044E00090E02CC08C2F0E944522811126C0C4313F
:1044F000E1F070F4CB3081F0C031D1F40E94CE1FD6
:104500008CE197E00E944A0582E08093C60115C0C5
:10451000C93259F0C83361F489E297E00E944A0534
:1045200080E297E00E944A0508C01092C60104C1CB
:104530008AE197E00E944A05FFC081E08170FEC0D9
:10454000C43228F5CE3108F0C1C0CB30A1F1D0F48F
:10455000C73009F0D3C08EE18093120182E38093CB
:1045600011018AE08093100184E180930F0188E0BB
:1045700080930E0188E280930D0180EC95E00E940B
:104580004A05BFC0C33149F1C431C1F0B7C0CB3413
:1045900009F4A9C028F4C93289F0C83361F0AEC06B
:1045A000C13509F49EC0C23509F499C0CE3409F072
:1045B000A5C06AE09EC00E94CE1FA3C08091C50125
:1045C000882319F01092C5019CC08DEC95E00E94E3
:1045D0004A0581E08093C601B1C087EA95E00E9458
:1045E0004A0585E995E00E944A05809112011F92D3
:1045F0008F9382E995E09F938F930E94E30580E972
:1046000095E00E944A058EE795E00E944A05809158
:1046100011011F928F938BE795E09F938F930E94D8
:10462000E30589E795E00E944A058AE695E00E9445
:104630004A05809110011F928F9387E695E09F9322
:104640008F930E94E30585E695E00E944A0584E584
:1046500095E00E944A0580910F011F928F9381E59A
:1046600095E09F938F930E94E3058FE495E00E946D
:104670004A058AE395E00E944A0580910E011F9247
:104680008F9387E395E09F938F930E94E30585E3E3
:1046900095E00E944A058EE195E00E944A058091CE
:1046A0000D011F928F938BE195E09F938F930E9452
:1046B000E30589E195E00E944A058DB79EB74896CB
:1046C0000FB6F8949EBF0FBE8DBF1BC0CE51EC2F0E
:1046D000F0E0E95DFE4F80818093C50112C061E08A
:1046E00003C061E006C06AE08091C5010E94E51F39
:1046F00008C08091C5010E94882003C08EEB95E020
:1047000013C08091C501882369F01F928F9388EBB5
:1047100095E09F938F930E94E3050F900F900F9069
:104720000F9004C085EB95E00E944A0581E006C029
:104730001092C60180E002C080E000CFCF910895C2
:104740000E94A7236894B1110C94362408950E9406
:104750001B2488F09F5798F0B92F9927B751B0F0D4
:10476000E1F0660F771F881F991F1AF0BA95C9F7F5
:1047700014C0B13091F00E943524B1E008950C943A
:104780003524672F782F8827B85F39F0B93FCCF3ED
:10479000869577956795B395D9F73EF49095809572
:1047A000709561957F4F8F4F9F4F0895E89409C092
:1047B00097FB3EF490958095709561957F4F8F4F54
:1047C0009F4F9923A9F0F92F96E9BB279395F6956A
:1047D000879577956795B795F111F8CFFAF4BB0FE8
:1047E00011F460FF1BC06F5F7F4F8F4F9F4F16C04C
:1047F000882311F096E911C0772321F09EE8872FD6
:10480000762F05C0662371F096E8862F70E060E091
:104810002AF09A95660F771F881FDAF7880F96950A
:10482000879597F9089557FD9058440F551F59F0F3
:104830005F3F71F04795880F97FB991F61F09F3F8D
:1048400079F087950895121613061406551FF2CFB6
:104850004695F1DF08C0161617061806991FF1CF06
:1048600086957105610508940895E894BB2766272D
:104870007727CB0197F908950E944F240C94C02408
:104880000E94B22438F00E94B92420F0952311F040
:104890000C94A9240C94AF2411240C9436240E9467
:1048A000132470F3959FC1F3950F50E0551F629F3D
:1048B000F001729FBB27F00DB11D639FAA27F00D79
:1048C000B11DAA1F649F6627B00DA11D661F829FA0
:1048D0002227B00DA11D621F739FB00DA11D621F85
:1048E000839FA00D611D221F749F3327A00D611DA2
:1048F000231F849F600D211D822F762F6A2F112484
:104900009F5750409AF0F1F088234AF0EE0FFF1FB6
:10491000BB1F661F771F881F91505040A9F79E3F0D
:10492000510580F00C94A9240C9436245F3FE4F3E5
:10493000983ED4F3869577956795B795F795E79563
:104940009F5FC1F7FE2B880F911D9695879597F96C
:10495000089597F99F6780E870E060E008959FEF01
:1049600080EC089500240A94161617061806090606
:10497000089500240A9412161306140605060895D5
:10498000092E0394000C11F4882352F0BB0F40F45D
:10499000BF2B11F460FF04C06F5F7F4F8F4F9F4F9D
:1049A0000895991B79E004C0991F961708F0961B8B
:1049B000881F7A95C9F78095089597FB072E16F4FE
:1049C000009407D077FD09D00E94F72407FC05D09A
:1049D0003EF4909581959F4F0895709561957F4F16
:1049E0000895EE0FFF1F0590F491E02D0994AA1B86
:1049F000BB1B51E107C0AA1FBB1FA617B70710F0CA
:104A0000A61BB70B881F991F5A95A9F780959095FB
:0A4A1000BC01CD010895F894FFCF1A
:104A1A008508760953091F09EB0801AC0128081417
:104A2A000A321E404D362270032303ED02CB025791
:104A3A000270028902A2020102030405060708099C
:024A4A0000006A
:106800000000000000000000040005000600070072
:10681000080009000A000B000C000D000E000F001C
:1068200010001100120013001400150016001700CC
:10683000180019001A001B001C001D001E001F007C
:10684000200021002200230024002500260027002C
:10685000280000002A002B002C002D002E002F0005
:10686000300031A1320033003400350036003700EB
:106870003800E00000000000000000000000000000
:106880000000000000000000000000000000000008
:1068900000000000000000000000000000004F00A9
:1068A000500051005200530067005400550056003C
:1068B000580059005A005B005C005D005E005F00FC
:1068C0006000610062006300640000005700000087
:1068D00000000000000000000000000000000000B8
:1068E00000000000000000000000000000000000A8
:1068F0000000E100E200E300000000000000F1A160
:106900000100010001000100EA4401000100E2442D
:106910000100010001000100460001004A004B0097
:10692000010001004700480001000100E9440100A6
:106930000100010001000100010001003A003B00DC
:106940003C003D003E003F0040004100420043004B
:10695000010000004C00010001004400450052000D
:1069600049000100010050004F0029004D004E0079
:1069700051000100010001000100010001000100BF
:1069800001000100010001000100010001000100FF
:1069900001000100010001000100010001004D00A3
:1069A0004A004E004B0001000100010001000100FF
:1069B00001000100010001000100010001000100CF
:1069C00001000100010001000100010001000100BF
:1069D00001000100010001000100010001000100AF
:1069E000010001000100010001000100010001009F
:1069F000010001000100010001000100010001008F
:00000001FF
